:100000000C9437000C945F000C945F000C945F001C
:100010000C945F000C945F000C945F000C944C02F5
:100020000C945F000C945F000C945F000C945F00D4
:100030000C945F000C945F000C945F000C945F00C4
:100040000C945F000C945F000C945F000C945F00B4
:100050000C945F000C945F000C945F000C945F00A4
:100060000C945F000C945F009B004502C0031124B8
:100070001FBECFEFD4E0DEBFCDBF11E0A0E0B1E006
:10008000ECEEFDE002C005900D92A431B107D9F766
:1000900011E0A4E1B1E001C01D92AF3AB107E1F770
:1000A00010E0CEE6D0E004C02297FE010E94F106E7
:1000B000C836D107C9F70E94A2000C94F5060C942B
:1000C00000000F931F93019799F56F5F7F4F81F5A4
:1000D00020E042E064E484E191E00E94920120E0AB
:1000E00043E064E48CE191E00E9492010CE211E0B3
:1000F0002CED35E041E064E171E084E291E00E94A2
:10010000B9042CED35E040E06CE171E084E391E06E
:100110000E94B90420E042E063E484E491E00E949C
:10012000440120E043E063E48CE491E00E94440158
:100130001F910F9108956FEF7FEF81E090E00E9493
:1001400061000895CF92DF92EF92FF920F931F9379
:10015000CF93DF930E94DE0168EE73E00E94850278
:1001600084E2C82E81E0D82EC4E3D1E00E94DE01F3
:100170000E94E7017B018C0180914B018823B9F13A
:10018000E0914501F0914601208130E080914401E9
:1001900090E028233923232B51F161E07FEFC60142
:1001A0000E945B0461E07FEFCE010E945B040E942D
:1001B000DE0128EE33E0B801A7010E94F301882395
:1001C00061F36FEF70E0C6010E945B0461E07FEFB6
:1001D000CE010E945B040E94DE012CED35E0B801E7
:1001E000A7010E94F301882309F045C0EACF80915E
:1001F00053018823B1F1E0914D01F0914E0120812E
:1002000030E080914C0190E028233923232B49F1E1
:1002100061E07FEFC6010E945B0461E07FEFCE01E9
:100220000E945B040E94DE0128EE33E0B801A701C2
:100230000E94F301882361F361E07FEFC6010E9411
:100240005B046FEF70E0CE010E945B040E94DE0150
:100250002CED35E0B801A7010E94F301882359F481
:10026000EBCF6FEF70E0C6010E945B046FEF70E0B0
:10027000CE010E945B040E94DE01A801970164E1A7
:1002800070E00E94190272CF1F93CF93DF93EC01AD
:10029000122F0E94A4058F81882381F0CE010E9435
:1002A0002206EB81FC819881112321F08081892B2A
:1002B000808304C08081909598239083DF91CF91B3
:1002C0001F9108951F93CF93DF93EC01122F0E948B
:1002D000A4058F81882381F0CE010E942206EB8144
:1002E000FC819881112321F08081892B808304C0B7
:1002F0008081909598239083DF91CF911F910895ED
:10030000FC018781882369F0A381B48190816623F1
:1003100021F08C91892B8C9308958C919095982342
:100320009C9308951F93CF93DF93EC01122F0E94AB
:10033000A4058F81882339F0CE010E943306612FF6
:10034000CE010E948001DF91CF911F9108951F93EC
:10035000CF93DF93EC01122F0E94A4058F81882395
:1003600039F0CE010E943306612FCE010E94800138
:10037000DF91CF911F9108951092B200E0EBF0E071
:1003800080818260808380818E7F8083E1EBF0E0DA
:100390008081877F808380818460808380818D7F5E
:1003A000808380818E7F80838DE78093B300E0E738
:1003B000F0E08081826080837894089584E591E004
:1003C00008950E94BC0108950E94BC0108952FB7B2
:1003D000F894609155017091560180915701909168
:1003E00058012FBF0895EF92FF920F931F937A0148
:1003F0008B016FB7F8948091550190915601A091AF
:100400005701B09158016FBF60E070E08E199F09ED
:10041000A00BB10B40E050E0281739074A075B07F3
:1004200010F461E070E0CB011F910F91FF90EF900D
:100430000895EF92FF920F931F9379018A01AB0108
:1004400060E070E02FB7F8948091550190915601CB
:10045000A0915701B09158012FBF8E199F09A00B91
:10046000B10B481759076A077B0760F71F910F9177
:10047000FF90EF900895019739F46F5F7F4F21F45B
:1004800084E591E00E94E40108956FEF7FEF81E041
:1004900090E00E943B0208951F920F920FB60F92B8
:1004A00011242F933F934F935F936F937F938F9379
:1004B0009F93AF93BF93EF93FF93809155019091DA
:1004C0005601A0915701B09158010196A11DB11D8F
:1004D0008093550190935601A0935701B093580112
:1004E0000E9493020E94C703FF91EF91BF91AF91C9
:1004F0009F918F917F916F915F914F913F912F913C
:100500000F900FBE0F901F901895EFB7F8942091A1
:100510005501309156014091570150915801EFBF5C
:100520000E941902089589E591E00895DC012FB732
:10053000F89480E090E0FC01EE0FFF1FEE0FFF1F2C
:10054000E80FF91FEA0FFB1F13821282118210823B
:10055000848301968031910571F7A05BBF4F1D9296
:100560001D92FD0110821182128213822FBF089505
:10057000DC012FB7F89480E090E0FC01EE0FFF1F44
:10058000EE0FFF1FE80FF91FEA0FFB1F1382128205
:1005900011821082848301968031910571F7A05BEE
:1005A000BF4F1D921D92FD01108211821282138293
:1005B0002FBF0895EF92FF920F931F93CF93DF9376
:1005C000EC018B01BA01FFB6F894C05BDF4F588194
:1005D000C055D04020E0852F90E0FC01EE0FFF1FBA
:1005E000EE0FFF1FE80FF91FEC0FFD1F82819381B3
:1005F000892B39F02F5F203109F4B0C051505F7062
:10060000EACF503108F0AAC0DE01AF5ABF4F8C913B
:1006100090E0FC01EE0FFF1FEE0FFF1FE80FF91F28
:10062000EC0FFD1F82819381892B09F48FC08C917F
:1006300090E0FC01EE0FFF1FEE0FFF1FE80FF91F08
:10064000EC0FFD1F808191816817790708F47EC047
:10065000EC9022C08D919C91119768177907E0F07A
:10066000FD01848190E08217930711F4E42E14C0F9
:10067000FD018481E42E482F242F30E0D901AA0FF8
:10068000BB1FAA0FBB1FA20FB31FAC0FBD1FFD01E5
:1006900082819381892BF1F6852F90E0DC01AA0FEE
:1006A000BB1FAA0FBB1FA80FB91FAC0FBD1FFD01B9
:1006B0001383028311967C936E935483FFEFEF169E
:1006C00021F12E2D30E0F901EE0FFF1FEE0FFF1F7D
:1006D000E20FF31FEC0FFD1F848190E08217930758
:1006E00021F08481FD01848305C0CF5ADF4F5883F8
:1006F000C155D040F901EE0FFF1FEE0FFF1FE20FB3
:10070000F31FEC0FFD1F548329C09E01205B3F4F58
:10071000F901808190E0FC01EE0FFF1FEE0FFF1F3B
:10072000E80FF91FEC0FFD1F82819381892B29F0BF
:10073000F9018081FD01848305C0CF5ADF4F5883C2
:10074000C155D040C05BDF4F588308C0C05BDF4F4E
:100750004881C055D040EE24EA948ECFFFBEDF9191
:10076000CF911F910F91FF90EF900895019739F469
:100770006F5F7F4F21F489E591E00E94B8020895F0
:100780006FEF7FEF81E090E00E94B60308958F92B3
:100790009F92AF92BF92CF92DF92EF92FF920F9310
:1007A0001F93CF93DF935C010E94DE010E94E7015B
:1007B0009B01AC01F501EE5AFF4F80819181A2812E
:1007C000B38179018A01E81AF90A0A0B1B0B09F4B3
:1007D0004BC080819181A281B381281739074A07D4
:1007E0005B0728F40894E108F10801091109208346
:1007F000318342835383F501E05BFF4FC0804F019B
:1008000024C0DC8088819981A0E0B0E0E816F90678
:100810000A071B0788F0EA81FB811B821A82198272
:100820001882CC82D401DC92A081B1812D913C91BF
:10083000CF01F901099506C0888199818E199F0918
:1008400099838883CD1481F0CD2C8C2D90E0EC0120
:10085000CC0FDD1FCC0FDD1FC80FD91FCA0DDB1D4C
:100860008A819B81892B69F6DF91CF911F910F912E
:10087000FF90EF90DF90CF90BF90AF909F908F90C0
:100880000895FC018781882369F0A381B481908158
:10089000662321F08C91892B8C9308958C919095EF
:1008A00098239C93089561E00E948001089560E080
:1008B0000E9480010895CF92DF92EF92FF920F93F2
:1008C0001F93CF93DF93EC010E945C066C018C8137
:1008D000882309F443C0ED80FE800F8118850E94B3
:1008E000DE0124E130E0B801A7010E94F301882372
:1008F000A9F18B85882321F0D094C194D108D39499
:100900002C853D858E859F858C01020F131F281B2A
:10091000390B4FEF50E061E07FEFC6010E945505B3
:100920008C01FFB6F89489859A850E945304C8010A
:1009300064E170E00E948B06CB0168E070E00E94E9
:100940002C0589859A850E945704FFBE0E94DE010E
:100950000E94E7016D837E838F8398878A819B81C4
:10096000DF91CF911F910F91FF90EF90DF90CF908B
:100970000895AF92BF92DF92EF92FF920F931F9371
:10098000CF93DF93EC015B01D42E79010E944306E3
:1009900084E091E099838883DB86FD86EC861F875F
:1009A0000E87F5018781882389F0BA86A986C5015B
:1009B0000E9457040E94DE010E94E7016D837E833E
:1009C0008F839887CE010E94580602C01A86198626
:1009D000DF91CF911F910F91FF90EF90DF90BF902B
:1009E000AF900895AF92BF92DF92EF92FF920F9374
:1009F0001F93CF93DF93EC015B01D42E79010E940A
:100A0000430684E091E099838883DB86FD86EC864B
:100A10001F870E87F5018781882389F0BA86A9860A
:100A2000C5010E9457040E94DE010E94E7016D8308
:100A30007E838F839887CE010E94580602C01A8653
:100A40001986DF91CF911F910F91FF90EF90DF906A
:100A5000BF90AF9008950895CF93DF93CDB7DEB7E1
:100A600022970FB6F894DEBF0FBECDBF9A8389835D
:100A700089819A819C01629FC001639F900D729F42
:100A8000900D112403C089819A8101979A838983EB
:100A900089819A81892BB9F722960FB6F894DEBF27
:100AA0000FBECDBFDF91CF9108954F925F926F92AD
:100AB0007F928F929F92AF92BF92CF92DF92EF92EE
:100AC000FF920F931F932B015A0139017801E21A0B
:100AD000F30A0027F7FC0095102F9C01261B370B0B
:100AE000442737FD4095542FC801B7010E946C067A
:100AF000A418B508CC24B7FCC094DC2CA601950141
:100B00000E949E06882477FC8094982C620E731EA7
:100B1000841E951EC3011F910F91FF90EF90DF90EF
:100B2000CF90BF90AF909F908F907F906F905F908D
:100B30004F900895681779070CF4BC0146175707C2
:100B40000CF4BA01CB010895FC0181E090E002C0F1
:100B5000880F991F4A95E2F7808381E08783643488
:100B600019F165342CF4623449F0633451F511C045
:100B7000633679F06436C1F0623619F584E290E0AC
:100B80009683858383E290E09283818385E290E07F
:100B900015C087E290E09683858386E290E0928399
:100BA000818388E290E00AC08AE290E096838583A0
:100BB00089E290E0928381838BE290E09483838347
:100BC000089517820895FC0181E090E002C0880F2B
:100BD000991F4A95E2F7808381E08783643419F195
:100BE00065342CF4623449F0633451F511C0633636
:100BF00079F06436C1F0623619F584E290E09683AC
:100C0000858383E290E09283818385E290E015C042
:100C100087E290E09683858386E290E092838183E9
:100C200088E290E00AC08AE290E09683858389E2B8
:100C300090E0928381838BE290E094838383089594
:100C400017820895CF93DF93DC01EC018F81882315
:100C500039F0ED81FE8190818C918095892380838C
:100C6000DF91CF910895CF93DF93DC01EC018F8169
:100C7000882331F0ED81FE8180819C91892B8083D6
:100C8000DF91CF910895FC018EE091E09183808304
:100C90001382128214820895FC018EE091E0918308
:100CA00080831382128214820895FC0114820895B5
:100CB00021E0FC01248308950F931F938C01CB0145
:100CC0004FEF50E061E07FEF0E949A05F8019383B7
:100CD00082831F910F910895629FD001739FF0014D
:100CE000829FE00DF11D649FE00DF11D929FF00DBC
:100CF000839FF00D749FF00D659FF00D9927729FF3
:100D0000B00DE11DF91F639FB00DE11DF91FBD017D
:100D1000CF011124089597FB092E07260AD077FDED
:100D200004D027D006D000201AF4709561957F4F2B
:100D30000895F6F7909581959F4F089597FB092E9A
:100D400005260ED057FD04D028D00AD0001C38F458
:100D500050954095309521953F4F4F4F5F4F0895E7
:100D6000F6F790958095709561957F4F8F4F9F4FC7
:100D70000895AA1BBB1B51E107C0AA1FBB1FA617E2
:100D8000B70710F0A61BB70B881F991F5A95A9F734
:100D900080959095BC01CD010895A1E21A2EAA1B61
:100DA000BB1BFD010DC0AA1FBB1FEE1FFF1FA2171B
:100DB000B307E407F50720F0A21BB30BE40BF50B18
:100DC000661F771F881F991F1A9469F760957095A1
:100DD000809590959B01AC01BD01CF010895EE0F68
:0C0DE000FF1F0590F491E02D0994FFCF57
:100DEC00000000005B0458065506000000002B05AF
:040DFC00580655063A
:00000001FF
